:020000040000FA
:0A0000000000000029EF00F039D0E5
:0800180076D09EA8FED7AD6E64
:1000200012000C6A0B6EFF0E0B260C2200D0D8A01B
:100030001200030E0A6EE60E02D8F5D70A6AFE0F0A
:10004000096EE86A0A5AD8A012000000090600D01A
:10005000F8D7006A4F0EAF6EB06A240EAC6E900EE9
:10006000AB6E00010F0EC16E070EB46EC69A400E45
:10007000926EE00E936EC00E946E59D09EAA17D069
:10008000ABA404D0AE50AE50AB881100ABA205D0EB
:10009000AE50AE50AB98AB8811002D2A00EE39F06F
:1000A0002D50E926000EEA22AECFEFFF1100F2A498
:1000B00009D0F294114A122AD6CF0FF0D7CF10F000
:1000C000817A11002D502E5C0AE02E2A00EE39F0C4
:1000D0002E50E926000EEA22EF50146E01D014686B
:1000E0001200396A2D6A2E6A9D8A9F8AF28EF28CDE
:1000F00012009D9A396A2D6A2E6AAE50AE50AB98A6
:10010000AB889D8A1200F29EE0CF4DF4D8CF4EF41A
:10011000E8CF4FF4F28E0001A192F29E4DC4E0FFB1
:100120004EC4D8FF4FC4E8FFF28E10001000CB6819
:10013000BE6A0C0EBD6E9494BB6ABA6E9492050EA4
:10014000CA6E7F0ECB6EBE6A0C0EBD6E9494BB6AF7
:10015000BA6E949292908990929289929294899494
:100160009296899692988998939A8A9A94988B985D
:10017000949A8B9A94908B9093948A94CF0EBD16F8
:10018000000EBD12000EBE6ECF0EBA16000EBA12D1
:10019000000EBB6E236A36EC06F030EC08F0320E2F
:1001A00040DF939A8A9A94988B98949A8B9A949019
:1001B0008B909290899093948A94286802EE39F0FB
:1001C000140EEE68E82EFDD7276A23908ADF91DFB0
:1001D000CD6AF294F28A870ED56EB16AA192A0829E
:1001E000D08EA292B00EB16E01EE39F0010EF46E17
:1001F000F36AF306000EF45AEE6AF450F310F9E1D4
:100200002F6A306AD6CF0FF0D7CF10F05BDF14C063
:1002100013F0B90E135C09E3FE0E135C03E34CEF1D
:1002200003F003D0166A4CEF03F013AE22D0166A27
:10023000880E135C05E113C016F01768186817D014
:10024000980E135C05E113C016F019681A680FD0F8
:10025000A80E135C05E113C016F01B681C6807D0DC
:10026000B80E135C04E113C016F01D681E684AEF57
:1002700003F0165203E14CEF03F00CD2880E165C2B
:10028000D8A475D0172803E113C017F06FD013C09E
:1002900018F0180E175C02E1899267D0190E175CEE
:1002A00002E1899462D01A0E175C02E189965DD052
:1002B0001B0E175C02E1899858D0210E175C0CE3E5
:1002C0006D0E175C09E223A006D0880EA6DE17503B
:1002D000A4DE1850A2DE49D0730E175C0CE37D0E2D
:1002E000175C09E223A006D0880E97DE175095DE32
:1002F000185093DE3AD00C0E175C07E1CF0EBD16F6
:10030000000EBD12000EBE6E30D00D0E175C07E160
:10031000CF0EBA16000EBA12000EBB6E26D00E0E0D
:10032000175C0AE1279002013C693B693A69396927
:1003300031808B98000119D00F0E175C0AE12792CB
:10034000020140693F693E693D6931808B9A000135
:100350000CD0100E175C08E1279402014469436930
:100360004269416931808B900001176893D1980EE2
:10037000165CD8A478D1192803E113C019F072D102
:1003800013C01AF01A52D8A46DD0210E195C0CE3D8
:100390006D0E195C09E223A006D0980E3EDE1950BE
:1003A0003CDE1A503ADE5DD0720E195C0CE37D0E15
:1003B000195C09E223A006D0980E2FDE19502DDE1D
:1003C0001A502BDE4ED0180E195C02E1899249D0EA
:1003D000190E195C02E1899444D01A0E195C02E1ED
:1003E00089963FD01B0E195C02E189983AD00C0E19
:1003F000195C07E1CF0EBD16000EBD12000EBE6ED9
:1004000030D00D0E195C07E1CF0EBA16000EBA12ED
:10041000000EBB6E26D00E0E195C0AE12790020179
:100420003C693B693A69396931808B98000119D080
:100430000F0E195C0AE12792020140693F693E698B
:100440003D6931808B9A00010CD0100E195C08E1D7
:1004500027940201446943694269416931808B9064
:100460000001FFD0210E195C0FE36D0E195C0CE248
:1004700023A009D0980E0DEC00F019500DEC00F0FF
:100480001A500DEC00F0EDD0730E195C0FE37D0EE9
:10049000195C0CE223A009D0980E0DEC00F0195065
:1004A0000DEC00F01A500DEC00F0DBD00C0E195CD6
:1004B00016E1036A1AC002F0D890023603360236FB
:1004C000033600EE02F0CF0EBD16EE38300BBD1233
:1004D000ED30F36EEF30BE6EF332BE32C2D00D0E91
:1004E000195C16E1036A1AC002F0D890023603368E
:1004F0000236033600EE02F0CF0EBA16EE38300B9D
:10050000BA12ED30F36EEF30BB6EF332BB32A9D0CE
:100510000E0E195C2FE18B8827807F0E1A5C20E27B
:1005200002EE4DF0D8901A34E926000EEA22EECF02
:1005300006F0EFCF07F006500F24026E0750102090
:10054000036E000E1120046E000E1220056E05C011
:100550003CF204C03BF203C03AF202C039F205D0CB
:1005600002013C693B693A69396900011AC034F0FB
:10057000318077D00F0E195C2FE18B8A27827F0E96
:100580001A5C20E202EE4DF0D8901A34E926000EF3
:10059000EA22EECF06F0EFCF07F006500F24026EEE
:1005A00007501020036E000E1120046E000E122062
:1005B000056E05C040F204C03FF203C03EF202C027
:1005C0003DF205D0020140693F693E693D69000185
:1005D0001AC035F0318045D0100E195C2FE18B80A8
:1005E00027847F0E1A5C20E202EE4DF0D8901A3478
:1005F000E926000EEA22EECF06F0EFCF07F0065014
:100600000F24026E07501020036E000E1120046E9E
:10061000000E1220056E05C044F204C043F203C070
:1006200042F202C041F205D00201446943694269C5
:10063000416900011AC036F0318013D0180E195CE0
:1006400002E189820ED0190E195C02E1898409D079
:100650001A0E195C02E1898604D01B0E195C01E1B7
:100660008988196817D0A80E165C09E11B2803E1D8
:1006700013C01BF003D013C01CF019D90BD0B80E57
:10068000165C08E11D2803E113C01DF003D013C060
:100690001EF0F4D931B0D0D8050E285CD8B0BCD04B
:1006A00029500F5C2A5010582B5011582C501258BA
:1006B000D8A0B1D02C8E28522DE127B008D002014D
:1006C0003C693B693A6939698B98000122D0345002
:1006D000156E02EE4DF0D8901534E926000EEA2290
:1006E000EECF06F0EFCF07F006500F24026E075052
:1006F0001020036E000E1120046E000E1220056EF5
:1007000005C03CF204C03BF203C03AF202C039F229
:10071000827880D0010E285C2DE127B208D002013A
:1007200040693F693E693D698B9A000122D035508E
:10073000156E02EE4DF0D8901534E926000EEA222F
:10074000EECF06F0EFCF07F006500F24026E0750F1
:100750001020036E000E1120046E000E1220056E94
:1007600005C040F204C03FF203C03EF202C03DF2B9
:10077000827A50D0020E285C2DE127B408D0020105
:1007800044694369426941698B90000122D0365027
:10079000156E02EE4DF0D8901534E926000EEA22CF
:1007A000EECF06F0EFCF07F006500F24026E075091
:1007B0001020036E000E1120046E000E1220056E34
:1007C00005C044F204C043F203C042F202C041F249
:1007D000827020D0030E285C12E1B80E0DEC00F000
:1007E000420E0DEC00F0400E0DEC00F023808A84E8
:1007F0000201486947694669456900010BD0040E4A
:10080000285C07E123928B9002014C694B694A698D
:100810004969000111D80DD012AE0BD0126A116ACD
:10082000106A0F6A02EE39F0140EEE68E82EFDD75A
:10083000276A817202EF01F028682C8E156A050E76
:10084000155C33E2D8901534E96EEA6AEA36E93687
:10085000EA36390EE926020EEA22EFCF02F0ECCF9B
:1008600003F0ECCF04F0ECCF05F02950025C2A50E5
:1008700003582B5004582C50055815E2D8901534C5
:10088000E96EEA6AEA36E936EA36390EE926020EF8
:10089000EA22EFCF29F0ECCF2AF0ECCF2BF0ECCF0F
:1008A0002CF015C028F0152ACAE331901200210E51
:1008B0001B5C0FE36D0E1B5C0CE223A009D0A80E9D
:1008C0000DEC00F01B500DEC00F01C500DEC00F096
:1008D000D3D0760E1B5C0FE3800E1B5C0CE223A0D2
:1008E00009D0A80E0DEC00F01B500DEC00F01C50D0
:1008F0000DEC00F0C1D00C0E1B5C16E1336A1CC07D
:1009000032F0D890323633363236333600EE32F0AB
:10091000CF0EBD16EE38300BBD12ED30F36EEF305A
:10092000BE6EF332BE32A8D00D0E1B5C16E1336AE8
:100930001CC032F0D890323633363236333600EEC1
:1009400032F0CF0EBA16EE38300BBA12ED30F36E2D
:10095000EF30BB6EF332BB328FD00E0E1B5C2DE13D
:1009600027A022D002EE4DF0D8901C34E926000ECC
:10097000EA22EECF06F0EFCF07F006500F24026E0A
:1009800007501020036E000E1120046E000E12207E
:10099000056E05C03CF204C03BF203C03AF202C04F
:1009A00039F21CC034F006D002013C693B693A6957
:1009B00039698B98000131805FD00F0E1B5C2DE1EF
:1009C00027A222D002EE4DF0D8901C34E926000E6A
:1009D000EA22EECF06F0EFCF07F006500F24026EAA
:1009E00007501020036E000E1120046E000E12201E
:1009F000056E05C040F204C03FF203C03EF202C0E3
:100A00003DF21CC035F006D0020140693F693E69E5
:100A10003D698B9A000131802FD0100E1B5C2CE1B8
:100A200027A422D002EE4DF0D8901C34E926000E07
:100A3000EA22EECF06F0EFCF07F006500F24026E49
:100A400007501020036E000E1120046E000E1220BD
:100A5000056E05C044F204C043F203C042F202C076
:100A600041F21CC036F006D0020144694369426974
:100A700041698B90000131801B6812001D520FE00C
:100A8000080E1D5C0CE223A009D0B80E0DEC00F09E
:100A90001D500DEC00F01E500DEC00F0A7D00D0E17
:100AA0001D5C0CE123A009D0B80E0DEC00F01D5028
:100AB0000DEC00F01E500DEC00F098D0100E1D5CF7
:100AC0000FE3400E1D5C0CE223A009D0B80E0DEC24
:100AD00000F01D500DEC00F01E500DEC00F086D023
:100AE000420E1D5CD8A452D01E5226E123A009D08C
:100AF000B80E0DEC00F0420E0DEC00F0000E0DEC07
:100B000000F0FF0E0F24026EFF0E1020036E000E89
:100B10001120046E000E1220056E05C04CF204C0B8
:100B20004BF203C04AF202C049F223902382929012
:100B300089908A947CD829D023B225D023B019D0AB
:100B4000FF0E0F24026EFF0E1020036E000E112008
:100B5000046E000E1220056E05C048F204C047F274
:100B600003C046F202C045F23180929089808B909A
:100B700009D0B80E0DEC00F0420E0DEC00F07F0E27
:100B80000DEC00F002D08A948B8030D0430E1D5CB7
:100B90000FE3720E1D5C0CE223A009D0B80E0DEC21
:100BA00000F01D500DEC00F01E500DEC00F01ED0BA
:100BB0007B0E1D5C0DE123A009D0B80E0DEC00F0FA
:100BC0007B0E0DEC00F01E500DEC00F011D80ED095
:100BD0007C0E1D5C0BE123A009D0B80E0DEC00F0DB
:100BE0007C0E0DEC00F01E500DEC00F01D681200A4
:100BF00002013C693B693A69396940693F693E696C
:100C00003D69446943694269416931808B988B9A97
:100C10008B900001CF0EBA16000EBA12000EBB6EFA
:100C2000CF0EBD16000EBD12000EBE6E12000201E8
:100C30003C693B693A69396940693F693E693D6988
:100C4000446943694269416931808B988B9A8B90E2
:100C50000001CF0EBA16000EBA12000EBB6ECF0EF8
:100C6000BD16000EBD12000EBE6E1200E90E02018E
:100C7000506FF80E4F6F740E526FFC0E516F4D0E89
:100C8000546FFD0E536F3A0E566F7E0E556F2E0E3B
:100C9000586FCB0E576F260E5A6F5969210E5C6F35
:100CA0006D0E5B6F1D0E5E6F3F0E5D6F190E606FF8
:100CB0005F69170E626F660E616F150E646F450EE9
:100CC000636F130E666F7F0E656F110E686F676935
:100CD000100E6A6FB60E696F0F0E6C6F990E6B6F08
:100CE0000E0E6E6F9F0E6D6F0D0E706FC30E6F6FD9
:100CF0000D0E726F716B0C0E746F500E736F0B0EC6
:100D0000766FB30E756F0B0E786F240E776F0A0E29
:100D10007A6FA30E796F0A0E7C6F2C0E7B6F090E13
:100D20007E6FC00E7D6F090E806F5C0E7F6F090EA7
:100D3000826F816B080E846FAA0E836F080E866F18
:100D40005B0E856F080E886F110E876F070E8A6F16
:100D5000CD0E896F070E8C6F8C0E8B6F070E8E6F0A
:100D6000500E8D6F070E906F170E8F6F060E926FDD
:100D7000E20E916F060E946FAF0E936F060E966F94
:100D8000800E956F060E986F530E976F060E9A6F32
:100D9000280E996F060E9C6F9B6B050E9E6FD90EE9
:100DA0009D6F050EA06FB50E9F6F050EA26F920E80
:100DB000A16F050EA46F710EA36F050EA66F510EE5
:100DC000A56F050EA86F330EA76F050EAA6F160E3E
:100DD000A96F040EAC6FFA0EAB6F040EAE6FE00E8F
:100DE000AD6F040EB06FC60EAF6F040EB26FAE0ED5
:100DF000B16F040EB46F960EB36F040EB66F800E13
:100E0000B56F040EB86F6A0EB76F040EBA6F550E49
:100E1000B96F040EBC6F410EBB6F040EBE6F2E0E79
:100E2000BD6F040EC06F1B0EBF6F040EC26F090EA4
:100E3000C16F030EC46FF70EC36F030EC66FE60ECD
:100E4000C56F030EC86FD60EC76F030ECA6FC60EEE
:100E5000C96F030ECC6FB70ECB6F030ECE6FA80E0B
:100E6000CD6F030ED06F990ECF6F030ED26F8C0E25
:100E7000D16F030ED46F7E0ED36F030ED66F710E3B
:100E8000D56F030ED86F640ED76F030EDA6F580E4E
:100E9000D96F030EDC6F4C0EDB6F030EDE6F400E5E
:100EA000DD6F030EE06F340EDF6F030EE26F290E6D
:100EB000E16F030EE46F1F0EE36F030EE66F140E77
:100EC000E56F030EE86F0A0EE76F030EEA6FE96B3A
:100ED000020EEC6FF60EEB6F020EEE6FED0EED6F85
:100EE000020EF06FE30EEF6F020EF26FDA0EF16F8B
:100EF000020EF46FD20EF36F020EF66FC90EF56F8D
:100F0000020EF86FC10EF76F020EFA6FB80EF96F8E
:100F1000020EFC6FB00EFB6F020EFE6FA90EFD6F8E
:100F2000020E0301006FA10E0201FF6F020E03010A
:100F3000026F9A0E016F020E046F920E036F020E83
:100F4000066F8B0E056F020E086F840E076F020E80
:100F50000A6F7D0E096F020E0C6F760E0B6F020E7C
:100F60000E6F700E0D6F020E106F690E0F6F020E76
:100F7000126F630E116F020E146F5D0E136F020E6F
:100F8000166F570E156F020E186F510E176F020E67
:100F90001A6F4B0E196F020E1C6F460E1B6F020E5E
:100FA0001E6F400E1D6F020E206F3A0E1F6F020E55
:100FB000226F350E216F020E246F300E236F020E4A
:100FC000266F2B0E256F020E286F260E276F020E3E
:100FD0002A6F210E296F020E2C6F1C0E2B6F020E32
:100FE0002E6F170E2D6F020E306F120E2F6F020E26
:100FF000326F0D0E316F020E346F090E336F020E19
:10100000366F040E356F020E386F376B010E3A6F74
:10101000FC0E396F010E3C6FF70E3B6F010E3E6FF9
:10102000F30E3D6F010E406FEF0E3F6F010E426FEA
:10103000EB0E416F010E446FE70E436F010E466FDA
:10104000E30E456F010E486FDF0E476F010E4A6FCA
:10105000DB0E496F010E4C6FD80E4B6F0001120072
:1010600003014E6B4D6B0A0E506F170E4F6F020E41
:10107000156E0001800E155C20E21504086E03EE6B
:101080004DF0D8900834E926000EEA22EECF06F0A3
:10109000EFCF07F06F0E0624026E000E0720036EDE
:1010A00003EE4DF0D8901534E926000EEA2202C076
:0E10B000EEFF03C0EFFF152ADCE31200FFD7AE
:020000040030CA
:0300010006170ED1
:020005008580F4
:060008000FC00FE00F40E5
:00000001FF
